:020000040000FA
:020000009F2837
:080008007028820750344934CE
:100010004334313436344634383434342D34303487
:10002000343420345234543443343134333430345F
:10003000323472342E34613473346D3420343034BD
:10004000313430343734303435340D340A344C34B0
:100050004D343334333435342034313430346D342A
:1000600056342F34B0344B340D340A3441344434D4
:10007000433420344134443437343834393436341A
:100080000D340A34443461346C346C346134733468
:100090002034443453343134333430343234203423
:1000A00068346F3472346C346F34673465342034A0
:1000B0005234543443340D340A34523453343234C9
:1000C00033343234203434343834303430342C3413
:1000D00038342C344E342C3432340D340A34003459
:1000E000A200030EA30083010A08A5008A0183125F
:1000F0000408A4008B1C95280B1200008B10B00183
:10010000000006189228AF230830B100AA2303107C
:1001100006180314B00CB10B8628AF23AA23AA2318
:100120008B1095283F30C022B00124088400250898
:100130008A00230E8300A20E220E09000000031382
:1001400083168B0183120C3084008001840A841E84
:10015000A52883160030850015308600810181179F
:100160000113831200308500861200308C000520B8
:10017000FF390319BF28C0220C08013EB628D4233A
:1001800086162E22920112089522920AFF3903192F
:10019000CB28C022C3282E22D2238612BC219A1338
:1001A0009C137E21A721D4232E221115B00186167F
:1001B000D223BC21111DDE28F7212E220B168B170E
:1001C000D4238B130B12FF3030050319D828B0123B
:1001D0004D3030060319172941303006031907291D
:1001E0005330300603198612523030060319861632
:1001F000543030060319232B1111483030060319EF
:10020000052911112130C022D8281115D8288616A9
:100210009201911012089522920AFF3903191229AE
:10022000C0220A294B239114D2238616D8282E22C5
:100230001030920012089522920AFF3903192229E0
:10024000C0221A292E223730920012089522920AD3
:10025000FF3903192E29C0222529D223AD223008C7
:10026000C02231303006031D37294F227729303024
:100270003006031D3D295722772933303006031DF0
:1002800043295D22772932303006031D4929652232
:10029000772935303006031D4F296B2277293430FA
:1002A0003006031D55297322772937303006031D88
:1002B0005B297922772936303006031D6129812296
:1002C000772939303006031D67298722772938308E
:1002D0003006031D6D298F2277291B303006031D40
:1002E00073292E22D8282130C022B001D8287921A4
:1002F00022297E21F721B001D223080085110000B8
:1003000000000000000000000000051185148316A5
:10031000051183128E30D7210030D72107308F008E
:10032000803097001A30840085100000851100008D
:100330000000851400001708D7210008D721840A7F
:10034000970A970A8F0B94298510000008008511E1
:100350000000051100008514831605118312851411
:1003600000008E30D7210030D7219030D721AD301A
:10037000D72185100000080085118510831605110E
:10038000831200000000000005118514BF30D72142
:100390008316051583121A308400E721E721E7212F
:1003A000E721E721E721E7218510000008009900F7
:1003B00008308E008511191C05111918051500004B
:1003C000000000008515990C8E0BDA290800083012
:1003D0008D00851100000000800C80130519801726
:1003E0008515000000008D0BE929840A08002030E3
:1003F000C0222030C022BC213230C0223030C02286
:10040000012A20081E222F30C0221E081E222F3053
:10041000C0221D081E222030C0222030C0221C080D
:100420001E223A30C0221B081E223A30C0221A086F
:100430001E222030C0222030C02208008C008D00F7
:100440008C0E0F308C0530300C07C0220D088C004C
:100450000F308C0530300C07C02208000D30C02250
:100460000A30C02208000A308C002030C0228C0BD9
:10047000352A08008C00FE309B3E0C028C0D831C3C
:10048000FA3E0C1CA03E8C0C08008C0001300C02C3
:100490008C0D831CFA3E0C1CA03E8C0C08001B0823
:1004A000603C031908001B083A229B0008001B0847
:1004B0000319080045229B0008001C08243C03196E
:1004C00008001C083A229C0008001C0803190800B8
:1004D00045229C0008001D08283C031908001D083F
:1004E0003A229D0008001D080319080045229D00BE
:1004F00008001E08123C031908001E083A229E003C
:1005000008001E080319080045229E000800200864
:10051000993C0319080020083A22A000080020088E
:10052000031908004522A00008008900831608145A
:100530008312080808008B138B1B9C2A83165530E6
:100540008900AA30890088148818A42A0812831206
:1005500008008316081483120800B0010000061872
:10056000AF2AAF230830B100AA23031006180314E2
:10057000B00CB10BB42AAA2308002A30C02208000C
:10058000AF000830B1000510AA23AF0C0318CA2A27
:100590000510CB2A0514AA23B10BC52A0514AA23DA
:1005A00008004008BE004108BF00400EF038BA0005
:1005B000BA07E23EBB00323EBD0040080F39BB0720
:1005C000BB07BD07E93EBC00BC07BC07410E0F39A5
:1005D000BC07BD07BC0DBD0DBD09BD0D41080F39E0
:1005E000BD07BA0D0730B9000A30BD07BC03031CB4
:1005F000F52ABC07BB03031CF92ABB07BA03031C7B
:10060000FD2ABA07B903031C012B3A08303EC02269
:100610003B08303EC0223C08303EC022911C122BC9
:100620002C30C0223D08303EC022911C1E2B2E30A3
:10063000C0224330C0222030C02208006D30C022CA
:100640005630C0221B2B91140830920012089522BC
:10065000920AFF3903192E2BC022262B5323470859
:10066000C0004608C1000A30C200AA30C3004308D7
:10067000C1024208031C420FC0029113C01F442B49
:10068000C009C109C10A91174008C4004108C5004A
:10069000D1222E22D82853234708C0004608C10083
:1006A000D1222E22080086118610061A861200001A
:1006B0008614C601C701B4237523752375237523DA
:1006C000043093007523C70D061D47100619471403
:1006D000930B622B083093007523C60D061D461040
:1006E00006194614930B6C2B080086110000861522
:1006F00000000800031020309800AA01AB01AC01F3
:10070000AD01AE01A90DA80DA70DA60DAE0DAD0D45
:10071000AC0DAB0DAA0D980B8E2BA92B2E3084009F
:100720009E232D3084009E232C3084009E232B306A
:1007300084009E232A3084009E23822B03300007EE
:10074000A100A119800030300007A100A11B80008A
:10075000080008003A30B200B20BAC2B0800193088
:10076000B200B20BB12B08000130940001309500AB
:1007700004309600E12B01309400013095001230D6
:100780009600E12B0130940001309500B3309600C3
:10079000E12B0A309700970BCE2B0800C223CB2BFE
:1007A0001930CA2B6430CA2B03309400BB3095003B
:1007B00001309600E12B9700970BDF2B0800D42324
:1007C000DC2B960BE12B950BE12B940BE12B080016
:0E07D0004308C1024208031C420FC002080089
:02400E00F13F80
:1042000041346E3461346C346F3467343D3400347F
:10421000543465346D347034653472343D34003454
:104220004D346F3464346934663420345234543439
:1042300043340D340A342034203441344D344A346C
:1042400048344D340D340A342B3420343934373467
:104250003534333431340D340A342D342034383489
:1042600036343434323430340D340A340034433488
:10427000643465343D340034523445345334453469
:04428000543400347E
:00000001FF
